 Imath_dll

 Timestamp is 44d97f50 (Tue Aug 08 23:23:12 2006)

 Preferred load address is 10000000

 Start         Length     Name                   Class
 0001:00000000 00002ed8H .text                   CODE
 0001:00002ee0 000001b5H .text$yc                CODE
 0002:00000000 000000f4H .idata$5                DATA
 0002:000000f4 00000004H .CRT$XCA                DATA
 0002:000000f8 00000010H .CRT$XCU                DATA
 0002:00000108 00000004H .CRT$XCZ                DATA
 0002:0000010c 00000004H .CRT$XIA                DATA
 0002:00000110 00000004H .CRT$XIAA               DATA
 0002:00000114 00000004H .CRT$XIC                DATA
 0002:00000118 00000004H .CRT$XIZ                DATA
 0002:00000120 000008c8H .rdata                  DATA
 0002:000009e8 00000344H .rdata$r                DATA
 0002:00000d30 00000004H .rdata$sxdata           DATA
 0002:00000d34 00000004H .rtc$IAA                DATA
 0002:00000d38 00000004H .rtc$IMZ                DATA
 0002:00000d3c 00000004H .rtc$IZZ                DATA
 0002:00000d40 00000004H .rtc$TAA                DATA
 0002:00000d44 00000004H .rtc$TMZ                DATA
 0002:00000d48 00000004H .rtc$TZZ                DATA
 0002:00000d50 0000026cH .xdata$x                DATA
 0002:00000fbc 00000050H .idata$2                DATA
 0002:0000100c 00000014H .idata$3                DATA
 0002:00001020 000000f4H .idata$4                DATA
 0002:00001114 00000504H .idata$6                DATA
 0002:00001620 000000faH .edata                  DATA
 0003:00000000 000001ecH .data                   DATA
 0003:000001f0 00000498H .bss                    DATA

  Address         Publics by Value              Rva+Base       Lib:Object

 0000:00000000       __except_list              00000000     <absolute>
 0000:00000001       ___safe_se_handler_count   00000001     <absolute>
 0000:00009876       __ldused                   00009876     <absolute>
 0000:00009876       __fltused                  00009876     <absolute>
 0000:00000000       ___ImageBase               10000000     <linker-defined>
 0001:00000000       ?hsv2rgb_d@Imath@@YA?AV?$Vec3@N@1@ABV21@@Z 10001000 f   ImathColorAlgo.obj
 0001:00000190       ?hsv2rgb_d@Imath@@YA?AV?$Color4@N@1@ABV21@@Z 10001190 f   ImathColorAlgo.obj
 0001:00000330       ?rgb2hsv_d@Imath@@YA?AV?$Vec3@N@1@ABV21@@Z 10001330 f   ImathColorAlgo.obj
 0001:00000520       ?rgb2hsv_d@Imath@@YA?AV?$Color4@N@1@ABV21@@Z 10001520 f   ImathColorAlgo.obj
 0001:00000720       ?succf@Imath@@YAMM@Z       10001720 f   ImathFun.obj
 0001:000007c0       ?predf@Imath@@YAMM@Z       100017c0 f   ImathFun.obj
 0001:00000860       ?succd@Imath@@YANN@Z       10001860 f   ImathFun.obj
 0001:00000940       ?predd@Imath@@YANN@Z       10001940 f   ImathFun.obj
 0001:00000a20       ?length@?$Vec2@F@Imath@@QBEFXZ 10001a20 f   ImathVec.obj
 0001:00000ab0       ?normalize@?$Vec2@F@Imath@@QAEABV12@XZ 10001ab0 f   ImathVec.obj
 0001:00000ae0       ?normalizeExc@?$Vec2@F@Imath@@QAEABV12@XZ 10001ae0 f   ImathVec.obj
 0001:00000b60       ?normalizeNonNull@?$Vec2@F@Imath@@QAEABV12@XZ 10001b60 f   ImathVec.obj
 0001:00000b90       ?normalized@?$Vec2@F@Imath@@QBE?AV12@XZ 10001b90 f   ImathVec.obj
 0001:00000c20       ?normalizedExc@?$Vec2@F@Imath@@QBE?AV12@XZ 10001c20 f   ImathVec.obj
 0001:00000cf0       ?normalizedNonNull@?$Vec2@F@Imath@@QBE?AV12@XZ 10001cf0 f   ImathVec.obj
 0001:00000d80       ?length@?$Vec2@H@Imath@@QBEHXZ 10001d80 f   ImathVec.obj
 0001:00000df0       ?normalize@?$Vec2@H@Imath@@QAEABV12@XZ 10001df0 f   ImathVec.obj
 0001:00000e20       ?normalizeExc@?$Vec2@H@Imath@@QAEABV12@XZ 10001e20 f   ImathVec.obj
 0001:00000ea0       ?normalizeNonNull@?$Vec2@H@Imath@@QAEABV12@XZ 10001ea0 f   ImathVec.obj
 0001:00000ed0       ?normalized@?$Vec2@H@Imath@@QBE?AV12@XZ 10001ed0 f   ImathVec.obj
 0001:00000f60       ?normalizedExc@?$Vec2@H@Imath@@QBE?AV12@XZ 10001f60 f   ImathVec.obj
 0001:00001020       ?normalizedNonNull@?$Vec2@H@Imath@@QBE?AV12@XZ 10002020 f   ImathVec.obj
 0001:000010b0       ?length@?$Vec3@F@Imath@@QBEFXZ 100020b0 f   ImathVec.obj
 0001:00001150       ?normalize@?$Vec3@F@Imath@@QAEABV12@XZ 10002150 f   ImathVec.obj
 0001:00001180       ?normalizeExc@?$Vec3@F@Imath@@QAEABV12@XZ 10002180 f   ImathVec.obj
 0001:00001210       ?normalizeNonNull@?$Vec3@F@Imath@@QAEABV12@XZ 10002210 f   ImathVec.obj
 0001:00001240       ?normalized@?$Vec3@F@Imath@@QBE?AV12@XZ 10002240 f   ImathVec.obj
 0001:000012f0       ?normalizedExc@?$Vec3@F@Imath@@QBE?AV12@XZ 100022f0 f   ImathVec.obj
 0001:000013e0       ?normalizedNonNull@?$Vec3@F@Imath@@QBE?AV12@XZ 100023e0 f   ImathVec.obj
 0001:00001490       ?length@?$Vec3@H@Imath@@QBEHXZ 10002490 f   ImathVec.obj
 0001:00001510       ?normalize@?$Vec3@H@Imath@@QAEABV12@XZ 10002510 f   ImathVec.obj
 0001:00001540       ?normalizeExc@?$Vec3@H@Imath@@QAEABV12@XZ 10002540 f   ImathVec.obj
 0001:000015c0       ?normalizeNonNull@?$Vec3@H@Imath@@QAEABV12@XZ 100025c0 f   ImathVec.obj
 0001:000015f0       ?normalized@?$Vec3@H@Imath@@QBE?AV12@XZ 100025f0 f   ImathVec.obj
 0001:00001690       ?normalizedExc@?$Vec3@H@Imath@@QBE?AV12@XZ 10002690 f   ImathVec.obj
 0001:00001770       ?normalizedNonNull@?$Vec3@H@Imath@@QBE?AV12@XZ 10002770 f   ImathVec.obj
 0001:00001810       ??_GIntVecNormalizeExc@Imath@@UAEPAXI@Z 10002810 f i ImathVec.obj
 0001:00001810       ??_GNullVecExc@Imath@@UAEPAXI@Z 10002810 f i ImathVec.obj
 0001:00001810       ??_EIntVecNormalizeExc@Imath@@UAEPAXI@Z 10002810 f i ImathVec.obj
 0001:00001810       ??_ENullVecExc@Imath@@UAEPAXI@Z 10002810 f i ImathVec.obj
 0001:00001810       ??_GMathExc@Iex@@UAEPAXI@Z 10002810 f i ImathVec.obj
 0001:00001810       ??_EMathExc@Iex@@UAEPAXI@Z 10002810 f i ImathVec.obj
 0001:00001850       ??1IntVecNormalizeExc@Imath@@UAE@XZ 10002850 f i ImathVec.obj
 0001:00001850       ??1NullVecExc@Imath@@UAE@XZ 10002850 f i ImathVec.obj
 0001:00001880       ??0NullVecExc@Imath@@QAE@ABV01@@Z 10002880 f i ImathVec.obj
 0001:000018c0       ??0MathExc@Iex@@QAE@ABV01@@Z 100028c0 f i ImathVec.obj
 0001:00001900       ??$normalizeOrThrow@F@?A0xcd77a4ad@Imath@@YA_NAAV?$Vec3@F@1@@Z 10002900 f i ImathVec.obj
 0001:000019b0       ??$normalizeOrThrow@F@?A0xcd77a4ad@Imath@@YA_NAAV?$Vec2@F@1@@Z 100029b0 f i ImathVec.obj
 0001:00001a60       ??$normalizeOrThrow@H@?A0xcd77a4ad@Imath@@YA_NAAV?$Vec3@H@1@@Z 10002a60 f i ImathVec.obj
 0001:00001b10       ??$normalizeOrThrow@H@?A0xcd77a4ad@Imath@@YA_NAAV?$Vec2@H@1@@Z 10002b10 f i ImathVec.obj
 0001:00001bc0       ??0IntVecNormalizeExc@Imath@@QAE@ABV01@@Z 10002bc0 f i ImathVec.obj
 0001:00001c00       ??0BaseExc@Iex@@QAE@PBD@Z  10002c00 f   Iex_dll:Iex_dll.dll
 0001:00001c06       ?what@BaseExc@Iex@@UBEPBDXZ 10002c06 f   Iex_dll:Iex_dll.dll
 0001:00001c0c       ??0BaseExc@Iex@@QAE@ABV01@@Z 10002c0c f   Iex_dll:Iex_dll.dll
 0001:00001c12       ??1BaseExc@Iex@@UAE@XZ     10002c12 f   Iex_dll:Iex_dll.dll
 0001:00001c18       ??0?$basic_string@DU?$char_traits@D@std@@V?$allocator@D@2@@std@@QAE@ABV01@@Z 10002c18 f   msvcprt:MSVCP80.dll
 0001:00001c1e       ??0?$_String_val@DV?$allocator@D@std@@@std@@QAE@ABV01@@Z 10002c1e f   msvcprt:MSVCP80.dll
 0001:00001c30       __RTC_CheckEsp             10002c30 f   MSVCRT:stack.obj
 0001:00001c53       @_RTC_CheckStackVars@8     10002c53 f   MSVCRT:stack.obj
 0001:00001cb0       __ftol2_sse                10002cb0 f   MSVCRT:ftol2.obj
 0001:00001cb9       __ftol2_pentium4           10002cb9 f   MSVCRT:ftol2.obj
 0001:00001ccc       __ftol2_sse_excpt          10002ccc f   MSVCRT:ftol2.obj
 0001:00001ce6       __ftol2                    10002ce6 f   MSVCRT:ftol2.obj
 0001:00001d5c       _floor                     10002d5c f   MSVCRT:MSVCR80.dll
 0001:00001d62       __RTC_InitBase             10002d62 f   MSVCRT:init.obj
 0001:00001d88       __RTC_Shutdown             10002d88 f   MSVCRT:init.obj
 0001:00001d9a       __CIsqrt                   10002d9a f   MSVCRT:MSVCR80.dll
 0001:00001da0       __CxxThrowException@8      10002da0 f   MSVCRT:MSVCR80.dll
 0001:00001da6       ??_Etype_info@@UAEPAXI@Z   10002da6 f i MSVCRT:ti_inst.obj
 0001:00001df0       ??0exception@std@@QAE@ABV01@@Z 10002df0 f   MSVCRT:MSVCR80.dll
 0001:00001df6       ??3@YAXPAX@Z               10002df6 f   MSVCRT:MSVCR80.dll
 0001:00001e49       __CRT_INIT@12              10002e49 f   MSVCRT:crtdll.obj
 0001:000020fe       __DllMainCRTStartup@12     100030fe f   MSVCRT:crtdll.obj
 0001:000023bf       ?_RTC_Failure@@YAXPAXH@Z   100033bf f   MSVCRT:error.obj
 0001:000023f7       ?_RTC_StackFailure@@YAXPAXPBD@Z 100033f7 f   MSVCRT:error.obj
 0001:00002538       __get_sse2_info            10003538 f   MSVCRT:cpu_disp.obj
 0001:00002598       ___sse2_available_init     10003598 f   MSVCRT:cpu_disp.obj
 0001:000025a5       __RTC_SetErrorFuncW        100035a5 f   MSVCRT:userapi.obj
 0001:000025bc       ?_RTC_GetErrorFunc@@YAP6AHHPBDH00ZZPBX@Z 100035bc f   MSVCRT:userapi.obj
 0001:000025c2       ?_RTC_GetErrorFuncW@@YAP6AHHPB_WH00ZZPBX@Z 100035c2 f   MSVCRT:userapi.obj
 0001:000025c8       __CRT_RTC_INITW            100035c8 f   MSVCRT:MSVCR80.dll
 0001:000025ce       ?__ArrayUnwind@@YGXPAXIHP6EX0@Z@Z 100035ce f   MSVCRT:ehvecdtr.obj
 0001:0000262c       ??_M@YGXPAXIHP6EX0@Z@Z     1000362c f   MSVCRT:ehvecdtr.obj
 0001:0000268f       ___clean_type_info_names   1000368f f   MSVCRT:tncleanup.obj
 0001:0000269b       __onexit                   1000369b f   MSVCRT:atonexit.obj
 0001:0000273a       _atexit                    1000373a f   MSVCRT:atonexit.obj
 0001:0000274c       __RTC_Initialize           1000374c f   MSVCRT:initsect.obj
 0001:00002770       __RTC_Terminate            10003770 f   MSVCRT:initsect.obj
 0001:000027a0       __ValidateImageBase        100037a0 f   MSVCRT:pesect.obj
 0001:000027d0       __FindPESection            100037d0 f   MSVCRT:pesect.obj
 0001:00002812       __IsNonwritableInCurrentImage 10003812 f   MSVCRT:pesect.obj
 0001:0000287e       __initterm                 1000387e f   MSVCRT:MSVCR80.dll
 0001:00002884       __initterm_e               10003884 f   MSVCRT:MSVCR80.dll
 0001:0000288a       __amsg_exit                1000388a f   MSVCRT:MSVCR80.dll
 0001:00002890       ___CppXcptFilter           10003890 f   MSVCRT:MSVCR80.dll
 0001:00002896       _DllMain@12                10003896 f   MSVCRT:dllmain.obj
 0001:000028b8       __SEH_prolog4              100038b8 f   MSVCRT:sehprolg4.obj
 0001:000028fd       __SEH_epilog4              100038fd f   MSVCRT:sehprolg4.obj
 0001:00002911       __except_handler4          10003911 f   MSVCRT:chandler4gs.obj
 0001:00002934       ___security_init_cookie    10003934 f   MSVCRT:gs_support.obj
 0001:00002b1f       ?_RTC_GetSrcLine@@YAHPAEPA_WKPAH1K@Z 10003b1f f   MSVCRT:pdblkup.obj
 0001:00002d95       @__security_check_cookie@4 10003d95 f   MSVCRT:secchk.obj
 0001:00002da4       ?terminate@@YAXXZ          10003da4 f   MSVCRT:MSVCR80.dll
 0001:00002daa       ??1type_info@@UAE@XZ       10003daa f   MSVCRT:MSVCR80.dll
 0001:00002daa       ?_type_info_dtor_internal_method@type_info@@QAEXXZ 10003daa f   MSVCRT:MSVCR80.dll
 0001:00002db0       ___clean_type_info_names_internal 10003db0 f   MSVCRT:MSVCR80.dll
 0001:00002db6       __unlock                   10003db6 f   MSVCRT:MSVCR80.dll
 0001:00002dbc       ___dllonexit               10003dbc f   MSVCRT:MSVCR80.dll
 0001:00002dc2       __lock                     10003dc2 f   MSVCRT:MSVCR80.dll
 0001:00002dc8       __except_handler4_common   10003dc8 f   MSVCRT:MSVCR80.dll
 0001:00002dce       ___report_gsfailure        10003dce f   MSVCRT:gs_report.obj
 0001:00002ed2       __crt_debugger_hook        10003ed2 f   MSVCRT:MSVCR80.dll
 0002:00000000       __imp_?what@BaseExc@Iex@@UBEPBDXZ 10005000     Iex_dll:Iex_dll.dll
 0002:00000004       __imp_??0BaseExc@Iex@@QAE@ABV01@@Z 10005004     Iex_dll:Iex_dll.dll
 0002:00000008       __imp_??1BaseExc@Iex@@UAE@XZ 10005008     Iex_dll:Iex_dll.dll
 0002:0000000c       __imp_??0BaseExc@Iex@@QAE@PBD@Z 1000500c     Iex_dll:Iex_dll.dll
 0002:00000010       \177Iex_dll_NULL_THUNK_DATA 10005010     Iex_dll:Iex_dll.dll
 0002:00000014       __imp__SetUnhandledExceptionFilter@4 10005014     kernel32:KERNEL32.dll
 0002:00000018       __imp__UnhandledExceptionFilter@4 10005018     kernel32:KERNEL32.dll
 0002:0000001c       __imp__GetCurrentProcess@0 1000501c     kernel32:KERNEL32.dll
 0002:00000020       __imp__TerminateProcess@8  10005020     kernel32:KERNEL32.dll
 0002:00000024       __imp__VirtualQuery@12     10005024     kernel32:KERNEL32.dll
 0002:00000028       __imp__GetModuleFileNameW@12 10005028     kernel32:KERNEL32.dll
 0002:0000002c       __imp__GetProcessHeap@0    1000502c     kernel32:KERNEL32.dll
 0002:00000030       __imp__HeapAlloc@12        10005030     kernel32:KERNEL32.dll
 0002:00000034       __imp__HeapFree@12         10005034     kernel32:KERNEL32.dll
 0002:00000038       __imp__FreeLibrary@4       10005038     kernel32:KERNEL32.dll
 0002:0000003c       __imp__GetSystemTimeAsFileTime@4 1000503c     kernel32:KERNEL32.dll
 0002:00000040       __imp__GetCurrentProcessId@0 10005040     kernel32:KERNEL32.dll
 0002:00000044       __imp__GetCurrentThreadId@0 10005044     kernel32:KERNEL32.dll
 0002:00000048       __imp__GetTickCount@0      10005048     kernel32:KERNEL32.dll
 0002:0000004c       __imp__QueryPerformanceCounter@4 1000504c     kernel32:KERNEL32.dll
 0002:00000050       __imp__DisableThreadLibraryCalls@4 10005050     kernel32:KERNEL32.dll
 0002:00000054       __imp__LoadLibraryA@4      10005054     kernel32:KERNEL32.dll
 0002:00000058       __imp__GetProcAddress@8    10005058     kernel32:KERNEL32.dll
 0002:0000005c       __imp__MultiByteToWideChar@24 1000505c     kernel32:KERNEL32.dll
 0002:00000060       __imp__IsDebuggerPresent@0 10005060     kernel32:KERNEL32.dll
 0002:00000064       __imp__WideCharToMultiByte@32 10005064     kernel32:KERNEL32.dll
 0002:00000068       __imp__DebugBreak@0        10005068     kernel32:KERNEL32.dll
 0002:0000006c       __imp__RaiseException@16   1000506c     kernel32:KERNEL32.dll
 0002:00000070       __imp__InterlockedCompareExchange@12 10005070     kernel32:KERNEL32.dll
 0002:00000074       __imp__Sleep@4             10005074     kernel32:KERNEL32.dll
 0002:00000078       __imp__InterlockedExchange@8 10005078     kernel32:KERNEL32.dll
 0002:0000007c       \177KERNEL32_NULL_THUNK_DATA 1000507c     kernel32:KERNEL32.dll
 0002:00000080       __imp_??0?$basic_string@DU?$char_traits@D@std@@V?$allocator@D@2@@std@@QAE@ABV01@@Z 10005080     msvcprt:MSVCP80.dll
 0002:00000084       __imp_??0?$_String_val@DV?$allocator@D@std@@@std@@QAE@ABV01@@Z 10005084     msvcprt:MSVCP80.dll
 0002:00000088       \177MSVCP80_NULL_THUNK_DATA 10005088     msvcprt:MSVCP80.dll
 0002:0000008c       __imp____dllonexit         1000508c     MSVCRT:MSVCR80.dll
 0002:00000090       __imp___unlock             10005090     MSVCRT:MSVCR80.dll
 0002:00000094       __imp____clean_type_info_names_internal 10005094     MSVCRT:MSVCR80.dll
 0002:00000098       __imp_?_type_info_dtor_internal_method@type_info@@QAEXXZ 10005098     MSVCRT:MSVCR80.dll
 0002:0000009c       __imp_?terminate@@YAXXZ    1000509c     MSVCRT:MSVCR80.dll
 0002:000000a0       __imp____CppXcptFilter     100050a0     MSVCRT:MSVCR80.dll
 0002:000000a4       __imp___adjust_fdiv        100050a4     MSVCRT:MSVCR80.dll
 0002:000000a8       __imp___amsg_exit          100050a8     MSVCRT:MSVCR80.dll
 0002:000000ac       __imp___initterm_e         100050ac     MSVCRT:MSVCR80.dll
 0002:000000b0       __imp___lock               100050b0     MSVCRT:MSVCR80.dll
 0002:000000b4       __imp___decode_pointer     100050b4     MSVCRT:MSVCR80.dll
 0002:000000b8       __imp__free                100050b8     MSVCRT:MSVCR80.dll
 0002:000000bc       __imp___encoded_null       100050bc     MSVCRT:MSVCR80.dll
 0002:000000c0       __imp___malloc_crt         100050c0     MSVCRT:MSVCR80.dll
 0002:000000c4       __imp___encode_pointer     100050c4     MSVCRT:MSVCR80.dll
 0002:000000c8       __imp___CRT_RTC_INITW      100050c8     MSVCRT:MSVCR80.dll
 0002:000000cc       __imp_??3@YAXPAX@Z         100050cc     MSVCRT:MSVCR80.dll
 0002:000000d0       __imp_??0exception@std@@QAE@ABV01@@Z 100050d0     MSVCRT:MSVCR80.dll
 0002:000000d4       __imp___CxxThrowException@8 100050d4     MSVCRT:MSVCR80.dll
 0002:000000d8       __imp___CIsqrt             100050d8     MSVCRT:MSVCR80.dll
 0002:000000dc       __imp__floor               100050dc     MSVCRT:MSVCR80.dll
 0002:000000e0       __imp___except_handler4_common 100050e0     MSVCRT:MSVCR80.dll
 0002:000000e4       __imp___initterm           100050e4     MSVCRT:MSVCR80.dll
 0002:000000e8       __imp___crt_debugger_hook  100050e8     MSVCRT:MSVCR80.dll
 0002:000000ec       __imp___onexit             100050ec     MSVCRT:MSVCR80.dll
 0002:000000f0       \177MSVCR80_NULL_THUNK_DATA 100050f0     MSVCRT:MSVCR80.dll
 0002:000000f4       ___xc_a                    100050f4     MSVCRT:cinitexe.obj
 0002:00000108       ___xc_z                    10005108     MSVCRT:cinitexe.obj
 0002:0000010c       ___xi_a                    1000510c     MSVCRT:cinitexe.obj
 0002:00000118       ___xi_z                    10005118     MSVCRT:cinitexe.obj
 0002:00000130       __real@4018000000000000    10005130     ImathColorAlgo.obj
 0002:00000138       __real@3ff0000000000000    10005138     ImathColorAlgo.obj
 0002:00000140       __real@4010000000000000    10005140     ImathColorAlgo.obj
 0002:00000148       __real@4000000000000000    10005148     ImathColorAlgo.obj
 0002:000003c0       __real@3fe0000000000000    100053c0     ImathVec.obj
 0002:000003cc       ??_7NullVecExc@Imath@@6B@  100053cc     ImathVec.obj
 0002:000003d8       ??_7MathExc@Iex@@6B@       100053d8     ImathVec.obj
 0002:000003e4       ??_7IntVecNormalizeExc@Imath@@6B@ 100053e4     ImathVec.obj
 0002:000003f0       ??_7type_info@@6B@         100053f0     MSVCRT:ti_inst.obj
 0002:000003f4       __pDefaultRawDllMain       100053f4     MSVCRT:crtdll.obj
 0002:000003f4       __pRawDllMain              100053f4     MSVCRT:crtdll.obj
 0002:000003f8       ??_C@_0BO@GNIAFIKK@Unknown?5Runtime?5Check?5Error?6?$AN?$AA@ 100053f8     MSVCRT:error.obj
 0002:00000418       ??_C@_0CM@NGINOKPC@Stack?5memory?5around?5_alloca?5was?5@ 10005418     MSVCRT:error.obj
 0002:00000444       ??_C@_0DG@HKJMLLLP@A?5local?5variable?5was?5used?5before@ 10005444     MSVCRT:error.obj
 0002:0000047c       ??_C@_0BN@FFOINMNJ@Stack?5memory?5was?5corrupted?6?$AN?$AA@ 1000547c     MSVCRT:error.obj
 0002:000004a0       ??_C@_0BBN@GPMLNJCF@A?5cast?5to?5a?5smaller?5data?5type?5ha@ 100054a0     MSVCRT:error.obj
 0002:000005c0       ??_C@_0NN@NGPKDKPD@The?5value?5of?5ESP?5was?5not?5properl@ 100055c0     MSVCRT:error.obj
 0002:00000720       ??_C@_0CA@IODNCDPG@Run?9Time?5Check?5Failure?5?$CD?$CFd?5?9?5?$CFs?$AA@ 10005720     MSVCRT:error.obj
 0002:00000740       ??_C@_0BE@GNBOBNCK@Unknown?5Module?5Name?$AA@ 10005740     MSVCRT:error.obj
 0002:00000754       ??_C@_0BB@PFFGGCJP@Unknown?5Filename?$AA@ 10005754     MSVCRT:error.obj
 0002:00000768       ??_C@_1EA@NFKNIFJP@?$AAR?$AAu?$AAn?$AA?9?$AAT?$AAi?$AAm?$AAe?$AA?5?$AAC?$AAh?$AAe?$AAc?$AAk?$AA?5?$AAF?$AAa?$AAi?$AAl?$AAu?$AAr?$AAe?$AA?5?$AA?$CD?$AA?$CF?$AAd?$AA?5?$AA?9?$AA?5?$AA?$CF?$AAs?$AA?$AA@ 10005768     MSVCRT:error.obj
 0002:000007a8       ??_C@_1GM@OLMCBDMB@?$AAR?$AAu?$AAn?$AAt?$AAi?$AAm?$AAe?$AA?5?$AAC?$AAh?$AAe?$AAc?$AAk?$AA?5?$AAE?$AAr?$AAr?$AAo?$AAr?$AA?4?$AA?6?$AA?$AN?$AA?5?$AAU?$AAn?$AAa?$AAb?$AAl?$AAe?$AA?5?$AAt?$AAo@ 100057a8     MSVCRT:error.obj
 0002:00000814       ??_C@_0CG@IAFNJNEE@Stack?5corrupted?5near?5unknown?5var@ 10005814     MSVCRT:error.obj
 0002:0000083c       ??_C@_0BP@OGBCLIBO@Stack?5around?5_alloca?5corrupted?$AA@ 1000583c     MSVCRT:userapi.obj
 0002:0000085c       ??_C@_0CK@CNLNOEPB@Local?5variable?5used?5before?5initi@ 1000585c     MSVCRT:userapi.obj
 0002:00000888       ??_C@_0BI@CIGMDCBH@Stack?5memory?5corruption?$AA@ 10005888     MSVCRT:userapi.obj
 0002:000008a0       ??_C@_0CK@FEGOIOPB@Cast?5to?5smaller?5type?5causing?5los@ 100058a0     MSVCRT:userapi.obj
 0002:000008cc       ??_C@_0BJ@HEGAHDFO@Stack?5pointer?5corruption?$AA@ 100058cc     MSVCRT:userapi.obj
 0002:000008e8       ??_C@_0M@EKFFODEC@MSPDB80?4DLL?$AA@ 100058e8     MSVCRT:pdblkup.obj
 0002:000008f4       ??_C@_0BF@BMIHBHCA@EnvironmentDirectory?$AA@ 100058f4     MSVCRT:pdblkup.obj
 0002:0000090c       ??_C@_0CN@EAEOKKOC@SOFTWARE?2Microsoft?2VisualStudio?2@ 1000590c     MSVCRT:pdblkup.obj
 0002:0000093c       ??_C@_0M@HLOHPNFA@RegCloseKey?$AA@ 1000593c     MSVCRT:pdblkup.obj
 0002:00000948       ??_C@_0BB@HHEIPGME@RegQueryValueExA?$AA@ 10005948     MSVCRT:pdblkup.obj
 0002:0000095c       ??_C@_0O@DCOGKJGG@RegOpenKeyExA?$AA@ 1000595c     MSVCRT:pdblkup.obj
 0002:0000096c       ??_C@_0N@JJPEKNFO@ADVAPI32?4DLL?$AA@ 1000596c     MSVCRT:pdblkup.obj
 0002:0000097c       ??_C@_01KDCPPGHE@r?$AA@    1000597c     MSVCRT:pdblkup.obj
 0002:00000980       ??_C@_0BB@KCIACLNC@PDBOpenValidate5?$AA@ 10005980     MSVCRT:pdblkup.obj
 0002:000009a0       __load_config_used         100059a0     MSVCRT:loadcfg.obj
 0002:000009e8       ??_R4MathExc@Iex@@6B@      100059e8     ImathVec.obj
 0002:000009fc       ??_R3MathExc@Iex@@8        100059fc     ImathVec.obj
 0002:00000a0c       ??_R2MathExc@Iex@@8        10005a0c     ImathVec.obj
 0002:00000a2c       ??_R1A@?0A@EA@MathExc@Iex@@8 10005a2c     ImathVec.obj
 0002:00000a48       ??_R1A@?0A@EA@BaseExc@Iex@@8 10005a48     ImathVec.obj
 0002:00000a64       ??_R3BaseExc@Iex@@8        10005a64     ImathVec.obj
 0002:00000a74       ??_R2BaseExc@Iex@@8        10005a74     ImathVec.obj
 0002:00000a90       ??_R1M@?0A@EA@?$basic_string@DU?$char_traits@D@std@@V?$allocator@D@2@@std@@8 10005a90     ImathVec.obj
 0002:00000aac       ??_R3?$basic_string@DU?$char_traits@D@std@@V?$allocator@D@2@@std@@8 10005aac     ImathVec.obj
 0002:00000abc       ??_R2?$basic_string@DU?$char_traits@D@std@@V?$allocator@D@2@@std@@8 10005abc     ImathVec.obj
 0002:00000ad0       ??_R1A@?0A@EA@?$basic_string@DU?$char_traits@D@std@@V?$allocator@D@2@@std@@8 10005ad0     ImathVec.obj
 0002:00000aec       ??_R1A@?0A@EA@?$_String_val@DV?$allocator@D@std@@@std@@8 10005aec     ImathVec.obj
 0002:00000b08       ??_R3?$_String_val@DV?$allocator@D@std@@@std@@8 10005b08     ImathVec.obj
 0002:00000b18       ??_R2?$_String_val@DV?$allocator@D@std@@@std@@8 10005b18     ImathVec.obj
 0002:00000b28       ??_R1A@?0A@EA@_String_base@std@@8 10005b28     ImathVec.obj
 0002:00000b44       ??_R3_String_base@std@@8   10005b44     ImathVec.obj
 0002:00000b54       ??_R2_String_base@std@@8   10005b54     ImathVec.obj
 0002:00000b60       ??_R1A@?0A@EA@_Container_base@std@@8 10005b60     ImathVec.obj
 0002:00000b7c       ??_R3_Container_base@std@@8 10005b7c     ImathVec.obj
 0002:00000b8c       ??_R2_Container_base@std@@8 10005b8c     ImathVec.obj
 0002:00000b94       ??_R1M@?0A@EA@?$_String_val@DV?$allocator@D@std@@@std@@8 10005b94     ImathVec.obj
 0002:00000bb0       ??_R1M@?0A@EA@_String_base@std@@8 10005bb0     ImathVec.obj
 0002:00000bcc       ??_R1M@?0A@EA@_Container_base@std@@8 10005bcc     ImathVec.obj
 0002:00000be8       ??_R1A@?0A@EA@exception@std@@8 10005be8     ImathVec.obj
 0002:00000c04       ??_R3exception@std@@8      10005c04     ImathVec.obj
 0002:00000c14       ??_R2exception@std@@8      10005c14     ImathVec.obj
 0002:00000c1c       ??_R4NullVecExc@Imath@@6B@ 10005c1c     ImathVec.obj
 0002:00000c30       ??_R3NullVecExc@Imath@@8   10005c30     ImathVec.obj
 0002:00000c40       ??_R2NullVecExc@Imath@@8   10005c40     ImathVec.obj
 0002:00000c64       ??_R1A@?0A@EA@NullVecExc@Imath@@8 10005c64     ImathVec.obj
 0002:00000c80       ??_R4IntVecNormalizeExc@Imath@@6B@ 10005c80     ImathVec.obj
 0002:00000c94       ??_R3IntVecNormalizeExc@Imath@@8 10005c94     ImathVec.obj
 0002:00000ca4       ??_R2IntVecNormalizeExc@Imath@@8 10005ca4     ImathVec.obj
 0002:00000cc8       ??_R1A@?0A@EA@IntVecNormalizeExc@Imath@@8 10005cc8     ImathVec.obj
 0002:00000ce4       ??_R4type_info@@6B@        10005ce4     MSVCRT:ti_inst.obj
 0002:00000cf8       ??_R3type_info@@8          10005cf8     MSVCRT:ti_inst.obj
 0002:00000d08       ??_R2type_info@@8          10005d08     MSVCRT:ti_inst.obj
 0002:00000d10       ??_R1A@?0A@EA@type_info@@8 10005d10     MSVCRT:ti_inst.obj
 0002:00000d30       ___safe_se_handler_table   10005d30     <linker-defined>
 0002:00000d34       ___rtc_iaa                 10005d34     MSVCRT:initsect.obj
 0002:00000d3c       ___rtc_izz                 10005d3c     MSVCRT:initsect.obj
 0002:00000d40       ___rtc_taa                 10005d40     MSVCRT:initsect.obj
 0002:00000d48       ___rtc_tzz                 10005d48     MSVCRT:initsect.obj
 0002:00000d50       __TI8?AVNullVecExc@Imath@@ 10005d50     ImathVec.obj
 0002:00000d60       __CTA8?AVNullVecExc@Imath@@ 10005d60     ImathVec.obj
 0002:00000d84       __CT??_R0?AVNullVecExc@Imath@@@8??0NullVecExc@Imath@@QAE@ABV01@@Z68 10005d84     ImathVec.obj
 0002:00000da0       __CT??_R0?AVMathExc@Iex@@@8??0MathExc@Iex@@QAE@ABV01@@Z68 10005da0     ImathVec.obj
 0002:00000dbc       __CT??_R0?AVBaseExc@Iex@@@8??0BaseExc@Iex@@QAE@ABV01@@Z68 10005dbc     ImathVec.obj
 0002:00000dd8       __CT??_R0?AV?$basic_string@DU?$char_traits@D@std@@V?$allocator@D@2@@std@@@8??0?$basic_string@DU?$char_traits@D@std@@V?$allocator@D@2@@std@@QAE@ABV01@@Z2812 10005dd8     ImathVec.obj
 0002:00000df4       __CT??_R0?AV?$_String_val@DV?$allocator@D@std@@@std@@@8??0?$_String_val@DV?$allocator@D@std@@@std@@QAE@ABV01@@Z112 10005df4     ImathVec.obj
 0002:00000e10       __CT??_R0?AV_String_base@std@@@8112 10005e10     ImathVec.obj
 0002:00000e2c       __CT??_R0?AU_Container_base@std@@@8112 10005e2c     ImathVec.obj
 0002:00000e48       __CT??_R0?AVexception@std@@@8??0exception@std@@QAE@ABV01@@Z12 10005e48     ImathVec.obj
 0002:00000e64       __TI8?AVIntVecNormalizeExc@Imath@@ 10005e64     ImathVec.obj
 0002:00000e74       __CTA8?AVIntVecNormalizeExc@Imath@@ 10005e74     ImathVec.obj
 0002:00000e98       __CT??_R0?AVIntVecNormalizeExc@Imath@@@8??0IntVecNormalizeExc@Imath@@QAE@ABV01@@Z68 10005e98     ImathVec.obj
 0002:00000fbc       __IMPORT_DESCRIPTOR_Iex_dll 10005fbc     Iex_dll:Iex_dll.dll
 0002:00000fd0       __IMPORT_DESCRIPTOR_MSVCP80 10005fd0     msvcprt:MSVCP80.dll
 0002:00000fe4       __IMPORT_DESCRIPTOR_MSVCR80 10005fe4     MSVCRT:MSVCR80.dll
 0002:00000ff8       __IMPORT_DESCRIPTOR_KERNEL32 10005ff8     kernel32:KERNEL32.dll
 0002:0000100c       __NULL_IMPORT_DESCRIPTOR   1000600c     Iex_dll:Iex_dll.dll
 0003:00000010       ??_R0?AVMathExc@Iex@@@8    10007010     ImathVec.obj
 0003:0000002c       ??_R0?AVBaseExc@Iex@@@8    1000702c     ImathVec.obj
 0003:00000048       ??_R0?AV?$basic_string@DU?$char_traits@D@std@@V?$allocator@D@2@@std@@@8 10007048     ImathVec.obj
 0003:00000094       ??_R0?AV?$_String_val@DV?$allocator@D@std@@@std@@@8 10007094     ImathVec.obj
 0003:000000cc       ??_R0?AV_String_base@std@@@8 100070cc     ImathVec.obj
 0003:000000ec       ??_R0?AU_Container_base@std@@@8 100070ec     ImathVec.obj
 0003:00000110       ??_R0?AVexception@std@@@8  10007110     ImathVec.obj
 0003:0000012c       ??_R0?AVNullVecExc@Imath@@@8 1000712c     ImathVec.obj
 0003:0000014c       ??_R0?AVIntVecNormalizeExc@Imath@@@8 1000714c     ImathVec.obj
 0003:00000180       ??_R0?AVtype_info@@@8      10007180     MSVCRT:ti_inst.obj
 0003:00000198       ?_RTC_ErrorLevels@@3PAHA   10007198     MSVCRT:error.obj
 0003:000001d8       ___native_dllmain_reason   100071d8     MSVCRT:natstart.obj
 0003:000001dc       ___native_vcclrit_reason   100071dc     MSVCRT:natstart.obj
 0003:000001e4       ___security_cookie         100071e4     MSVCRT:gs_cookie.obj
 0003:000001e8       ___security_cookie_complement 100071e8     MSVCRT:gs_cookie.obj
 0003:000001f0       ?identity33d@Imath@@3V?$Matrix33@N@1@A 100071f0     ImathMatrixAlgo.obj
 0003:00000238       ?identity44d@Imath@@3V?$Matrix44@N@1@A 10007238     ImathMatrixAlgo.obj
 0003:000002b8       ?identity44f@Imath@@3V?$Matrix44@M@1@A 100072b8     ImathMatrixAlgo.obj
 0003:000002f8       ?identity33f@Imath@@3V?$Matrix33@M@1@A 100072f8     ImathMatrixAlgo.obj
 0003:00000324       ?wsprintffp@@3P6AHPADPBDZZA 10007324     MSVCRT:error.obj
 0003:00000330       ?__type_info_root_node@@3U__type_info_node@@A 10007330     MSVCRT:tncleanup.obj
 0003:0000066c       __adjust_fdiv              1000766c     <common>
 0003:00000670       ___native_startup_state    10007670     <common>
 0003:00000674       ___native_startup_lock     10007674     <common>
 0003:00000678       ___onexitend               10007678     <common>
 0003:0000067c       ___onexitbegin             1000767c     <common>
 0003:00000680       ___sse2_available          10007680     <common>
 0003:00000684       ___dyn_tls_init_callback   10007684     <common>

 entry point at        0001:000020fe

 Static symbols

 0001:00001dfc       _pre_c_init                10002dfc f   MSVCRT:crtdll.obj
 0001:00001fe8       ___DllMainCRTStartup       10002fe8 f   MSVCRT:crtdll.obj
 0001:0000211f       ?DebuggerProbe@@YAHK@Z     1000311f f   MSVCRT:error.obj
 0001:0000216f       ?DebuggerRuntime@@YAHKHPAXPB_W@Z 1000316f f   MSVCRT:error.obj
 0001:000021d1       ?failwithmessage@@YAXPAXHHPBD@Z 100031d1 f   MSVCRT:error.obj
 0001:000024e8       _has_osfxsr_set            100034e8 f   MSVCRT:cpu_disp.obj
 0001:000029c8       ?GetPdbDll@@YAPAUHINSTANCE__@@XZ 100039c8 f   MSVCRT:pdblkup.obj
 0001:00002ee0       ??__Eidentity33f@Imath@@YAXXZ 10003ee0 f   ImathMatrixAlgo.obj
 0001:00002f30       ??__Eidentity33d@Imath@@YAXXZ 10003f30 f   ImathMatrixAlgo.obj
 0001:00002f80       ??__Eidentity44f@Imath@@YAXXZ 10003f80 f   ImathMatrixAlgo.obj
 0001:00003010       ??__Eidentity44d@Imath@@YAXXZ 10004010 f   ImathMatrixAlgo.obj

 Exports

  ordinal    name

        1    ?identity33d@Imath@@3V?$Matrix33@N@1@A (class Imath::Matrix33<double> Imath::identity33d)
        2    ?identity33f@Imath@@3V?$Matrix33@M@1@A (class Imath::Matrix33<float> Imath::identity33f)
        3    ?identity44d@Imath@@3V?$Matrix44@N@1@A (class Imath::Matrix44<double> Imath::identity44d)
        4    ?identity44f@Imath@@3V?$Matrix44@M@1@A (class Imath::Matrix44<float> Imath::identity44f)
